:1000000050C0000068C0000066C0000064C000006E
:1000100062C0000060C000005EC000005CC0000064
:100020005AC0000058C0000056C0000054C0000074
:1000300052C0000050C000004EC000004CC0000084
:100040004AC0000048C0000046C0000044C0000094
:1000500042C0000040C000003EC000003CC00000A4
:100060003AC0000069C3000036C0000034C0000080
:1000700032C0000030C000002EC000002CC00000C4
:100080002AC0000028C0000026C0000024C00000D4
:1000900022C0000020C000001EC000001CC00000E4
:1000A000C40311241FBECFEFCDBFDFE3DEBF2CE3BF
:1000B000A0E0BCE301C01D92A838B207E1F710E050
:1000C000C1E5D0E003C02197FE01F8D5C035D107C6
:1000D000D1F7B9D30EC694CF00008093C4088091A5
:1000E000C30887FFFCCF8091C4080895282F30E013
:1000F000F901ED57F24B40814F3F09F450C089326E
:1001000058F4F901E85FF24BE081EE2329F0E13089
:1001100099F010F0E63020F1F901E65AF24BE08157
:10012000A0E2EA9FF0011124FC5F8081842321F189
:10013000611120C046830895F901EF5CF24B5081B4
:10014000533008F05F5F7091010A81E090E001C0D8
:10015000880F5A95EAF7809587238093010ADCCFB0
:1001600080E1E89FF0011124E05AF54F81818F7EF4
:100170008183D2CF458308952F5C324BD9018C9176
:10018000309771F08F3F61F07096E80FF11D9FB7C7
:10019000F8948081611107C0877F80839FBF089595
:1001A000F0E0E0E0F4CF8860F8CF8F929F92AF92BA
:1001B000BF92CF92DF92EF92FF920F93CF93DF9394
:1001C0008091853C893210F461E090DF80911C3C85
:1001D000882319F081FF0DC07894DF91CF910F91A2
:1001E000FF90EF90DF90CF90BF90AF909F908F9057
:1001F000089580FFF2CF80901E3C90901F3CA0900D
:10020000203CB090213CC12CD12C7601E0E094013F
:10021000A501B601C701A0E045D581F1217030E00C
:1002200040E050E060E070E080E090E03BD5D1F04D
:10023000B0E0A0E0E03370F4AE2FA695A695A695A9
:1002400080E2A89FD0011124A05FBB4F8E2F877042
:10025000A80FB11DCE2FD0E0CA5ED34C88899C91E7
:10026000892B8C939401A501B601C70101E0FFD44D
:1002700049015A016B017C01EF5FC9CF8090223C9C
:100280009090233CA090243CB090253CC12CD12CD4
:100290007601E0E29401A501B601C701A0E002D514
:1002A00009F49BCF217030E040E050E060E070E066
:1002B00080E090E0F7D4D1F0B0E0A0E0E03370F45B
:1002C000AE2FA695A695A69580E2A89FD0011124F1
:1002D000A05FBB4F8E2F8770A80FB11DCE2FD0E02F
:1002E000CA5ED34C88899C91892B8C939401A5017B
:1002F000B601C70101E0BBD449015A016B017C0181
:10030000EF5FC8CFCF93DF9390E0FC01ED57F24B46
:1003100020812F3F61F0FC01E65AF24BE08130E290
:10032000E39FF0011124FC5F613021F42183DF9110
:10033000CF9108958F5C924BEC01A881AF3F69F09B
:10034000CF014096A80FB92FB11D9FB7F894228313
:100350008C9188608C939FBFEACFB0E0A0E0F5CF8E
:1003600080911B3C811117C010921C3C10921D3CC7
:1003700010921E3C10921F3C1092203C1092213C87
:100380001092223C1092233C1092243C1092253C67
:1003900081E080931B3C8091E3058C7F90911A3C17
:1003A000892B8093E305911119C061E084E0AADFF5
:1003B00061E086E0A7DF8091C10884608093C10876
:1003C0008091C00881628093C0089091143C809114
:1003D000153C9093C0088093C1080895913031F482
:1003E00061E08EE08FDF61E080E1E4CF923019F7C9
:1003F00061E08EE187DF61E080E2DCCF8FB7F894C7
:100400002091103C3091113C4091123C5091133C92
:10041000E091AA0AF091AB0A9091A60A90FF08C059
:100420002F5F3F4F4F4F5F4FE091AA0AF091AB0A09
:100430008FBFA8EEB3E00FD423E0F695E7952A9599
:10044000E1F76E0F7F1F811D911D08958F929F927E
:10045000AF92BF92CF92DF92EF92FF924B015C017D
:10046000CDDF6B017C01A8EEB3E0A5019401F3D3CD
:10047000C60ED71EE81EF91EC616D706E806F906F0
:1004800010F4BCDFF9CFBADF6C157D058E059F0532
:10049000D0F3FF90EF90DF90CF90BF90AF909F9000
:1004A0008F9008958F929F92AF92BF92CF92DF92DA
:1004B000EF92FF920F93CF93DF9380911C3C8823A0
:1004C00019F081FF19C0F89481E38093C00884E09B
:1004D0008093C1088091853C893208F098C060E023
:1004E000DF91CF910F91FF90EF90DF90CF90BF9071
:1004F000AF909F908F90FACD80FFE6CF80901E3C0A
:1005000090901F3CA090203CB090213CC12CD12C5D
:100510007601E0E09401A501B601C701A0E0C2D3D5
:1005200089F1217030E040E050E060E070E080E070
:1005300090E0B8D3D9F0B0E0A0E0E03370F4AE2F93
:10054000A695A695A69580E2A89FD0011124A05F4C
:10055000BB4F8E2F8770A80FB11DCE2FD0E08C918E
:10056000CA5ED34C888B8C91887F8C939401A501B3
:10057000B601C70101E07BD349015A016B017C013F
:10058000EF5FC8CF8090223C9090233CA090243C09
:10059000B090253CC12CD12C7601E0E29401A5015C
:1005A000B601C701A0E07ED309F48ECF217030E000
:1005B00040E050E060E070E080E090E073D3D9F07C
:1005C000B0E0A0E0E03370F4AE2FA695A695A69516
:1005D00080E2A89FD0011124A05FBB4F8E2F8770AF
:1005E000A80FB11DCE2FD0E08C91CA5ED34C888B62
:1005F0008C91887F8C939401A501B601C70101E01D
:1006000036D349015A016B017C01EF5FC7CFDF91FF
:10061000CF910F91FF90EF90DF90CF90BF90AF9070
:100620009F908F900895CF93C82F3CDF83E054DDD7
:100630008C2F52DD80E050DDC82FB7DD8C2FCF919D
:100640000895FF920F931F93CF93DF93C82FF62E39
:10065000172F042F27DF82E03FDD8C2F3DDDCF2DCC
:10066000D12F0C0F1D2F111DC017D10719F0899123
:1006700033DDFACFDF91CF911F910F91FF9095CD90
:100680001F93CF93DF93182FD62FC42F0BDF85E056
:1006900023DD812F21DD8D2F1FDD8C2F1DDDDF91CF
:1006A000CF911F9182CDCF92DF92EF92FF92CF93A5
:1006B000C82F482F60EE8FE0E3DF8FB7F894C0902B
:1006C000103CD090113CE090123CF090133C8FBF56
:1006D0008AE0C80ED11CE11CF11C2FB7F894809160
:1006E000103C9091113CA091123CB091133C2FBF53
:1006F0008C159D05AE05BF0578F48EE094DF807EF5
:10070000C813EBCF81E091E0892790E0CF91FF9073
:10071000EF90DF90CF90089580E0F5CFCF93DF93F7
:10072000D82FC62FBFDE82E0D7DC8D2FD5DC8C2FF3
:10073000D3DCDF91CF9139CD1F920F920FB60F927C
:1007400011248F939F93AF93BF938091103C90910E
:10075000113CA091123CB091133C0196A11DB11D1A
:100760008093103C9093113CA093123CB093133CA7
:1007700081E08093A60ABF91AF919F918F910F90D6
:100780000FBE0F901F901895CF93DF93E4E1FCE329
:10079000C4E0C18381E38083E6E1FCE31582148237
:1007A000DFDDD3E0D093853C61E083E0ABDDFDDCB1
:1007B000E5E5FCE385E190E080839183128213827A
:1007C00081E08483858326E130E0268337831086A9
:1007D0001186828792E0938727E130E0248735876E
:1007E00016861786808BD18B28E130E0228B338BE5
:1007F000148A158A868BC78B2CE130E0208F318FCD
:10080000128E138E848F95E0958F2BE130E0268F2A
:10081000378F10A211A282A396E093A32AE130E0C1
:1008200024A335A316A217A280A797E091A729E1D8
:1008300030E022A733A714A615A686A788E087A7CD
:10084000DF91CF910895CF93DF93CDB7DEB7A9970E
:10085000CDBFDEBF91E088ED84BF909361008091B1
:100860000206856080930206809100068160809375
:100870000006809102068F7C8065809302061092AC
:10088000E20582E08093E4059093030A8EEF809363
:10089000270A8093260A80E880932D0A80932B0AEA
:1008A0008093290A80932C0A80932A0A8093280A2D
:1008B00089E08093000A87E08093E505E0E8FAE0AC
:1008C00037E02EEF90E885E0318324879587808399
:1008D0007096E03C4AE0F407B9F71092A10A8FE362
:1008E0009FE18093AC0A9093AD0A8091A50A816044
:1008F0008093A50A1092A00A8091A00A816080933B
:10090000A00A78942DDD80916000806890E028ED49
:1009100024BF80936000C6DD80ECDEDB46DC6AE04D
:1009200070E080E090E092DDCE0101967C018EE0E7
:10093000D7011D928A95E9F74EE0B70180E381DE89
:100940004EE0B70180E47DDE4EE0B70180E579DE60
:1009500060E080E6E3DE60E080E7E0DE63EA8BE211
:10096000DDDE44E067E680E68BDE41E067E680E7B7
:1009700087DE8CE0E6EFFCE4DE011F9601900D922D
:100980008A95E1F74E01BFE08B0E911CD12CC12C52
:10099000A82C99A698E0B92EF401019111914F016C
:1009A00080E881DE892B61F40230110509F47BC0F7
:1009B000A0F501151105E1F10130110509F479C027
:1009C00080E871DE892B49F460E08AE2A7DE60E905
:1009D00089E2A4DE62E888E2A1DE80E064DE60ED08
:1009E00077E080E090E032DDA5E5CA2EACE3DA2EB8
:1009F000412C512C32014394FE017596EBA3FCA3CC
:100A0000FFE6CF16FDE3DF0609F064C000E010E06A
:100A100001151105E9F3F4DAFBCF0430110509F4EF
:100A200046C008F442C00530110551F688E101C006
:100A300080E0F1E0CF16D104F1F51E8E1D8EBC8E44
:100A40001B8E44E0BE01655E7F4FFBDD4FEFC41A95
:100A5000D40A86E0C816D10409F09ECF1F8E18A2D2
:100A600081E090E089A39AA38E01015E1F4F6E0181
:100A700093E2C90ED11C88E0B82ED8018D909D90CC
:100A80008D0180E810DE892B09F09ACF1E8E1D8E15
:100A9000BC8E1B8E8114910499F08A94892809F0E8
:100AA0008FCF84E20EC088E0C4CF80E1C2CF84E162
:100AB000C0CF84E0BECF1B8E1C8E1E8E1D8EC1CF7C
:100AC00080E244E0BE01655E7F4FBBDDC016D1060B
:100AD000A1F676CF4092003C5092013C6092023CDD
:100AE0007092033C44E04093043C87E48093083CCC
:100AF00091E19093093CA8E0A0930A3CB5E1B09342
:100B00000B3C86E0E2E0FDE4DE011F9601900D92D1
:100B10008A95E1F70A2D19A5F801819091908F012E
:100B20001401220C331CF101E80DF91DE455F24BC0
:100B3000B0808B2D78DD83FD87C01091043C193087
:100B400008F063C04091003C5091013C6091023C30
:100B50007091033CDB01CA018827B7FD8395992773
:100B6000AA27BB27282FDB01CA0188279927AA2794
:100B7000B0748DA39EA3AFA3B8A78FEF9FEFAFEF85
:100B8000BFE1211104C08FEF97E0A0E0B0E0842323
:100B90009523A623B723222309F446C08C839B8385
:100BA000CD01AA27BB27282F220F220F220F207E3C
:100BB000382F33703860232B2A8335E0969587953C
:100BC0003A95E1F789838DA19EA1AFA1B8A5892BA4
:100BD0008A2B8B2BB9F1812F80648D83412F50E0BC
:100BE00068E07CE3CE0106967BD045E0410FF10141
:100BF000E80DF91DE455F24BB701818122DD48E093
:100C000068E08B2D3DDD8B2D0EDD68EE73E080E01E
:100C100090E01CDCF6018081893210F462E072DB26
:100C2000F6E0CF0ED11CECCE9C0193E036952795D3
:100C30009A95E1F729838295880F807E8A831C82AA
:100C40001B82C1CF812FC9CFABA1BCA10A171B0743
:100C500009F062CFDACF38D0A59F900DB49F900DE8
:100C6000A49F800D911D1124089597FD1094002ECE
:100C7000083098F00850232F342F452F562F672F18
:100C8000782F892F912DF4CF159497958795779587
:100C9000679557954795379527950A95AAF7112493
:100CA000002D08950024A7FD00942A173005400563
:100CB000500560057005800590050895EE0FFF1F33
:100CC0000590F491E02D0994A29FB001B39FC0015B
:100CD000A39F01D0B29F700D811D1124911D089515
:100CE000FB01DC0102C001900D9241505040D8F749
:060CF0000895F894FFCF07
:100CF60000000100020003000400050000000100DE
:100D060002000000000000000000000000000005D6
:100D160001010101010100000000000000000000C7
:100D260000000000000000000203000001020304AE
:100D36000506070001020304050001020304050677
:100D46000700010203040506070001020300010271
:100D56000304050600000000000000000101010177
:100D66000101020202020202020203030303030359
:100D7600030304040404050505050505050102042D
:100D86000810204080010204081020010204081007
:100D9600204080010204081020408001020408015E
:0F0DA6000204081020403031364041465051566B
:00000001FF
